:200000000200A122FFFFFFFFFFFFFF02012B1200E47525FF7F01120248E4F525C201C20006
:20002000E4F52775260AE4F524E4F52302009ED292D2937F05120248C292A2B6E433FFBF58
:200040000102D201D292C2937F051200BCA2B6E433FFBF0102D200D29330031C752702E487
:20006000F526E4F524E4F523E52460FCE52470FC7526027525C880FE3001117525FF75279E
:2000800007E4F526E4F524E4F523801230000F752564752707752607E4F524E4F523020052
:2000A0002FE5A8C2AF549075812DA881760018B81FFAC0E0120003D0A802000E8F2BE4F5B4
:2000C0002C8017E4F52D7E007F09120228052D7D0AAF2DC3EF9D40EE052CAD2BAF2CC3EF6D
:2000E0009D40E022C2AFE4F589438901758CFF7EFE7F008F8AD2A9D28CD296D295D2B0D271
:20010000B3752196C203C204E4F528E4F525E4F522E4F524E4F523752707752607D292D207
:2001200093D290D29175970FD2AF22C003C004C005C006C007C0E0C0D053D0E7C28C758C47
:20014000FF7EFE7F008F8AD28CE5257004C202801774FF65257004D202800DE52260041503
:20016000228005852522B202300204B2B08002D2B0E528600415288041752832E5277004FE
:20018000D296801774FF65277004C296800DE524600415248005852724B296E5267004D274
:2001A00095801774FF65267004C295800DE523600415238005852623B2952004047B01805B
:2001C00002E4FBA2B3E433FFBF01047D018002E4FD7C00AF037E00EF5DFFEE5CFE4F600739
:2001E000D2047521968028A204E433FFBF01047B018002E4FB20B3047D018002E4FD7C00C4
:20020000AF037E00EF5DFFEE5CFE4F6002C204E521600415218002D203D0D0D0E0D007D0B6
:2002200006D005D004D00332C0A8C0E0C083C082C2AF8FE06009DFFEC3136003D5E0FDD09C
:2002400082D083D0E0D0A8228F29E4F52A80077F641200BC052AAD29AF2AC3EF9D40F0220D
:00000001FF
